:04000000B201CD2953
:100008000800B216B21EB212B2190E28B215472055
:10001800031835280830A3005B20A20DA30B102875
:10002800B21E402065206120B21A35203A202208ED
:100038000310C829B216B21EB21232192828FE3986
:10004800B30032150310C829321A3028A600321618
:1000580047200318352826084E2003183528B21ED5
:10006800C8294020652032113212B21136088400A6
:10007800340884178004462836088400340980052B
:100088008417800508003A20652040206120330845
:10009800B2190138A2000830A300A20D03183A20B3
:1000A800031C402065206120A30B51283A206520BD
:1000B8003608840034080005FF3E370884003509F7
:1000C80043283708840035083D2864007F2003183A
:1000D8006928CE20A8010830A300CF207F2003186C
:1000E800A80AAB1EA801A20CA30B7128AB1AA21375
:1000F800CF202208080036088400340884178004BA
:10010800841300052B1B3406FF3E0800A4002908B1
:100118000319C829C321A0002518831724088400BF
:10012800200880008313A40AA9038B280408A600CA
:10013800360884008030B3050830A7000310031880
:10014800B30AB420A60CA70BA3280000AB1A330CE3
:10015800B420CB210314B4202F08A3002E082F2984
:100168008413AB1FC328000834042B1F34068000F7
:10017800841700083404031C34068000CF280008C4
:100188003404031C34062B1B3406800084173409FE
:100198008005CF2833172B081F39003EA1002A08F5
:1001A8000E3E0318A10A331F3C293313A000023066
:1001B80060213C29B31329080319B3170430A80098
:1001C800250EEB202508EB20240EEB2024080F3900
:1001D800F63E0318073E0A3EF128A000A8030319BB
:1001E800B31329080319FB2828020318080020085C
:1001F800031DB313B31B0800303EC32983178001C6
:10020800840AFF3E031D0329C82921082004031975
:10021800A00A8030201AA1062019A106A018A1065C
:10022800210DA00DA10DC82903178D0083168C136D
:100238000C1483120C08C82903178C0083168C131E
:100248000C1555308D00AA308D008C148C182A2975
:100258000C11C829A301A200FF30A207031CA307A1
:10026800031CC8290330A100E6303C213029A10134
:10027800FC3EA000A109031C4729FF300000A0078D
:1002880003184229A0076400A10F41290800013E74
:10029800A7000A30A200A3019121A70B5029240826
:1002A80008000310A00DA10DFF3E031855292008D2
:1002B800C8290310A10CA00CFF3E03185D292008D3
:1002C800C829A101A301A20002307A29A301A20032
:1002D80003307A29A301A20001307A29A301A200E0
:1002E80006307A29A101A301A2000530A80023083D
:1002F8002102031D8129220820020430031801303D
:10030800031902302805031DFF30C8290038031DD2
:10031800FF300405031DFF30C829A501A4011030D2
:10032800A600210DA40DA50D2208A4022308031C74
:10033800230FA5020318A7292208A40723080318D6
:10034800230FA5070310A00DA10DA60B95292008C2
:10035800C8291030A800A101A001A70CA60C031CF5
:10036800BB292208A00723080318230FA107A10C03
:10037800A00CA50CA40CA80BB1292408C82984003A
:1003880031088A0030088200831303138312640043
:1003980008002030840060308A010321A0308400E6
:1003A80050308A0103211030840060308A01022114
:1003B8009030840060308A010221831607309F0044
:1003C800EE01EF01E301E201860187010510DB017F
:1003D800CE01C3010130CD00E801C430E700C201FD
:1003E80083120317900183160313CE01C301E8019A
:1003F800C430E7008312860107158716071487148F
:1004080005140130A300F4308A012F218316DB0183
:10041800AC011030AD00B401B50164005B08003CCC
:100428008A110A128312031D282A83160830BA007B
:100438000730B9002030AA00AB012030B200B30168
:1004480083128A110A12342A83160630BA0005303C
:10045800B9002830AA00AB012830B200B3018312DA
:10046800051064308A012E2105148A150A12D72C2A
:100478008A110A12632283165C0883128600871089
:10048800871607100711071507148A110A12632225
:1004980083165D08831286008710871607100711D8
:1004A800071507148A110A12632283165A08831241
:1004B8008600871607100711071507140800071488
:1004C8008316FF30860083128714071507108712DA
:1004D800003006180130A00001308A017621831609
:1004E800AE008312003086180130A00001308A0166
:1004F80076218316B0002E088312840083163008F4
:1005080083128A018A218A110A12031D632A871617
:10051800071483168601831208008A016322831652
:10052800FF308600831287108712071002308A0175
:100538003B2106088316C00083120714871683160A
:100548008601831208008A110A1255238A01912212
:10055800080083160130E8008312831626088312E8
:10056800A600831627088312A7002030A200A30143
:100578008A01AD218316AE00831225088316AF00C9
:100588002C08AE072D080318013EAF072408831274
:10059800A000831625088312A10083163A08831247
:1005A800A200A3018A0191218316B00083122108B9
:1005B8008316B1002E0830078312FB0083162F081C
:1005C8000318013E31078312FC007B088316A20042
:1005D80083127C088316A3002408CB002608CC00CD
:1005E80083127C088316DD0083127B088316DC00E7
:1005F8002430DA0083128A013C22640083166808DA
:10060800003C8A110A128312031D2E2B831624081C
:100618008312A000831625088312A10083163A08C6
:100628008312A200A3018A01912124088316AE0037
:10063800831225088316AF002E083902AE002F0951
:100648000318013EAF00F8302E04DA0083128A1135
:100658000A124F2B831624088312A000831625083C
:100668008312A10083163A088312A200A3018A010B
:10067800912124088316AE00831225088316AF0043
:100688002E083902AE002F090318013EAF00F030E2
:100698002E04DA0083128A0156228316E801831297
:1006A8000800831626088312A600831627088312DB
:1006B800A7002030A200A3018A01AD218316AE0055
:1006C800831225088316AF002C08AE072D080318DF
:1006D800013EAF0724088312A00083162508831261
:1006E800A10083163A088312A200A3018A0191216E
:1006F8008316B000831221088316B1002E08300734
:100708008312FB0083162F080318013E310783125A
:10071800FC007B088316A20083127C088316A300C2
:1007280083127C088316DD0083127B088316DC00A5
:100738002430DA0083128A013C2208008316580804
:100748005507A400A501A50D59085607A600A7013D
:10075800A70D83128A01B122831658085502A400F6
:10076800A501031CA50359085607A600A701A70D54
:1007780083128A01B122831655085807A400A501DF
:10078800A50D59085602A600A701031CA70383124A
:100798008A01B122831658085502A400A501031C3A
:1007A800A50359085602A600A701031CA703831234
:1007B8008A01B122831659085507A400A501A50D81
:1007C80058085607A600A701A70D83128A01B1226F
:1007D800831659085502A400A501031CA503560851
:1007E8005807A600A701A70D83128A01B122831614
:1007F80055085907A400A501A50D58085602A600DA
:10080800A701031CA70383128A01B1228316590882
:100818005502A400A501031CA50358085602A6000A
:10082800A701031CA70383128A01B12208008316BB
:1008380058085507A400A501A50D59085607A60094
:10084800A701A70D83128A01AD2283165808550205
:10085800A400A501031CA50359085607A600A70173
:10086800A70D83128A01AD22831655085807A400E4
:10087800A501A50D59085602A600A701031CA70348
:1008880083128A01AD22831658085502A400A501D7
:10089800031CA50359085602A600A701031CA703B9
:1008A80083128A01AD22831659085507A400A501B1
:1008B800A50D58085607A600A701A70D83128A019F
:1008C800AD22831659085502A400A501031CA503EF
:1008D80056085807A600A701A70D83128A01AD2262
:1008E800831655085907A400A501A50D58085602F6
:1008F800A600A701031CA70383128A01AD22831651
:1009080059085502A400A501031CA503580856025E
:10091800A600A701031CA70383128A01AD220800C1
:1009280083162D08DD002C08DC004230DA00831223
:100938008A013C2283162B08DD002A08DC0043309C
:10094800DA0083128A013C2283163508DD00340858
:10095800DC004030DA0083128A013C228316330817
:10096800DD003208DC004130DA0083128A013C22C3
:1009780083168030DA0083128A0156228316DD013D
:10098800DC012430DA0083128A013C228316983075
:10099800DA0083128A01562283160130C3008312BB
:1009A8006400F130831643028A110A128312031875
:1009B800FF2C83160130C600831264004130831671
:1009C80046028A110A1283120318F82C8316DD01D5
:1009D800C030DA0083128A0149228316C60A8A11B6
:1009E8000A128312031DE12C8316C30A8A110A1204
:1009F8008312031DD42C83169C30DA0083128A01DB
:100A0800562208008316D8015708D90083120230ED
:100A1800A600A701831657088312A200A3018A0122
:100A2800AD218316AE00831225088316AF002E0869
:100A3800023CA8002F08031C013E003CA9008312B9
:100A480064008316580859028A110A128312031C7B
:100A5800912D640003171008003C8A110A12031331
:100A6800031D3B2D8A01A2238A110A123D2D8A01FA
:100A78001B2464008A110A1283168310A91F831489
:100A880083128318652D0430A600A7018316580821
:100A98008312A200A3018A01AD218316AE0083123E
:100AA80025088316AF000630AE070318AF0A2E08D4
:100AB800A8072F080318013EA90783128A110A12F2
:100AC8008C2D831659085802AE00AF01031CAF03E2
:100AD80083120430A600A70183162E088312A200F1
:100AE80083162F088312A3008A01AD218316AE0056
:100AF800831225088316AF000A30AE070318AF0A21
:100B08002E08A8072F080318013EA907D903831246
:100B18008316D80A83128A01242D08008316D80167
:100B28005708D90083120230A600A7018316570878
:100B38008312A200A3018A01AD218316AE0083129D
:100B480025088316AF002E08023CA8002F08031CB6
:100B5800013E003CA900831264008316580859021C
:100B68008A110A128312031CF42D6400031710085B
:100B7800003C8A110A120313031DC72D8A01A22300
:100B88008A110A12C92D8A011B2483165908580292
:100B9800AE00AF01031CAF0383120430A600A70107
:100BA80083162E088312A20083162F088312A3002F
:100BB8008A01AD218316AE00831225088316AF0083
:100BC8000A30AE070318AF0A2E08A8072F08031823
:100BD800013EA9070330D902D80A83128A01B02D31
:100BE80008008A110A12232783164F085002C800EA
:100BF80052085302C9006400490848028A110A12BF
:100C08008312031C952E831649088312A000A101A4
:100C180002308A0158218316AE00831221088316F8
:100C2800AF0048082E02A8002F08031CFF3EA900A9
:100C38005208A600A70149088312A000A1010230AA
:100C48008A015821FD002108FE0083164808490240
:100C5800AE00AF01031CAF0383120230A600A70148
:100C680083162E088312A20083162F088312A3006E
:100C78008A01AD218316A000831225088316A100DE
:100C88004F08A400A5018312831624088312A0002C
:100C9800831625088312A1008316500883128A013F
:100CA8006E218A110A12031D942E64008A110A12F9
:100CB80083168310A91F831483128318702E7D084E
:100CC8008316A80783127E080318013E8316A90716
:100CD80083128A110A127B2E83162008A80721087E
:100CE8000318013EA907A60A0319A70A831264007C
:100CF80003171008003C8A110A120313031D892EDA
:100D08008A01B1228A110A128B2E8A01AD2283161A
:100D1800A40A0319A50A8A110A128312031D482E70
:100D28000800831648088312A000A10102308A0136
:100D380058218316AE00831221088316AF00490894
:100D48002E02A8002F08031CFF3EA9004F08A4008C
:100D5800A50148088312A000A10102308A01582188
:100D6800FD002108FE00831649084802AE00AF01C5
:100D7800031CAF0383120230A600A70183162E08B6
:100D88008312A20083162F088312A3008A01AD21C3
:100D98008316A000831225088316A1005208A60016
:100DA800A7018312831626088312A000831627083A
:100DB8008312A1008316530883128A016E218A11B7
:100DC8000A12031D222F64008A110A128316831047
:100DD800A91F831483128318FE2E7D088316A80783
:100DE80083127E080318013E8316A90783128A110D
:100DF8000A12092F83162008A80721080318013EA4
:100E0800A907A40A0319A50A831264000317100886
:100E1800003C8A110A120313031D172F8A01B122FD
:100E28008A110A12192F8A01AD228316A60A0319FC
:100E3800A70A8A110A128312031DD62E080064001D
:100E480083164F0850028A110A1283120318322F90
:100E580083164F085002CF07D0028312640083160E
:100E6800520853028A110A1283120318412F83165B
:100E780052085302D207D3028312080083162608A9
:100E88008312A000831627088312A1000830A2004D
:100E9800A3018A0191218316AE00831221088316CB
:100EA800AF002E088312A60083162F088312A7000E
:100EB8002030A200A3018A01AD218316AE0083125F
:100EC80025088316AF003408AE0735080318013E1D
:100ED800AF0724088312A000831625088312A100F7
:100EE80083163A088312A200A3018A01912183166E
:100EF800B000831221088316B1002E083007831230
:100F0800FB0083162F080318013E31078312FC00EB
:100F18007C088316DD0083127B088316DC002430EE
:100F2800DA0083128A013C2208008A150A12A920D5
:100F38008A013C228A150A125420203083163B026B
:100F4800BF0083128A01422783163F08DD00670825
:100F5800DA0083128A0149228A150A125E200800E3
:100F68007908A0007A08A10004308A014B21831671
:100F7800BB0083128A150A120E2008308316A407B4
:100F88000318A50A83127908A0007A08A100033083
:100F98008A014B218316BB0083128A150A120E2080
:100FA80008308316A4070318A50A83127908A0003D
:100FB8007A08A10002308A014B218316BB008312F4
:100FC8008A150A120E2008308316A4070318A50AEA
:100FD80083127908A0007A08A10001308A014B2108
:100FE8008316BB0083128A150A120E200830831656
:100FF800A4070318A50A83127908A0007A08A1009B
:1010080000308A014B218316BB0083128A150A120D
:101018000E20080083163B08093C8A150A12831221
:10102800031C2F288A150A121F208316CE0083124C
:101038008A150A122F2808308A0083163B08831263
:10104800820730343134323433343434353436343E
:10105800373438343934203083164E02BF008312B7
:101068008A01A62708008A150A12A9208A150A12D9
:1010780054208A01552383163E08DD006708DA00EC
:1010880083128A0149228A150A125E2008008A0101
:101098003C2283169830DA0083128A01562208000F
:1010A8008A150A12A92083169430DA0083128A015D
:1010B800562208008A150A12A92083169C30DA00E5
:1010C80083128A015622080083164308583E84007A
:1010D8000008AE008312FF30A200A20A22080F3CCB
:1010E8008A150A12031C9D288A150A12892083165C
:1010F8002E028A150A128312031D712822088316EC
:10110800DE0083128A150A129D2808308A002208F8
:10111800820730343134323433343434353436346D
:101128003734383439346134623463346434653480
:101138006634080083162D08DD002C08DC004230D8
:10114800DA0083128A013C22080083163508DD0084
:101158003408DC004030DA0083128A013C2208009F
:1011680083166B08A400A5016D08A600A7018312C9
:10117800831626088312A000831627088312A1006D
:1011880083166C0883128A016E218A150A12031DC0
:10119800E628640003171008003C8A150A12031396
:1011A800031DDB288A01B1228A150A12DD288A016B
:1011B800AD228316A60A0319A70A8A150A128312F2
:1011C800031DBC28013083166B07A400A501A50DDB
:1011D8006D08A600A7018312831626088312A000B3
:1011E800831627088312A10083166C0883128A01CC
:1011F8006E218A150A12031D20296400031710089E
:10120800003C8A150A120313031D0F298A01B12213
:101218008A150A1211298A01AD2283166908A607C0
:101228008A150A128312031CF0288316A70A8A1546
:101238000A128312031DF028080083166C08A60002
:10124800A7016B08A400A501831283162408831242
:10125800A000831625088312A10083166A0883124A
:101268008A016E218A150A12031D53296400031787
:101278001008003C8A150A120313031D48298A0125
:10128800B1228A150A124A298A01AD228316A40AB4
:101298000319A50A8A150A128312031D2929FF308A
:1012A80083166C07A600FF300318013EA7006B08E1
:1012B800A400A5018312831624088312A0008316B4
:1012C80025088312A10083166A0883128A016E21F9
:1012D8008A150A12031D8F29640003171008003CA1
:1012E8008A150A120313031D7E298A01B1228A1561
:1012F8000A1280298A01AD2283166908A4078A1573
:101308000A128312031C5F298316A50A8A150A127A
:101318008312031D5F2908008A01232783164F08BB
:10132800C300831264008316430850028A150A1208
:101338008312031CD42983165208C6008312640042
:101348008316460853028A150A128312031CCC29F5
:1013580083164308A400A5014608A600A701640057
:10136800831203171008003C8A150A120313031D81
:10137800C2298A01B1228A150A12C4298A01AD221A
:1013880083166908C6078A150A128312031CA32943
:1013980083166908C3078A150A128312031C962943
:1013A80008008A01232783164F08C30083126400AC
:1013B8008316430850028A150A128312031C192A3D
:1013C80083164308A400A5015208A600A7016400DB
:1013D800831203171008003C8A150A120313031D11
:1013E800FA298A01B1228A150A12FC298A01AD223A
:1013F80083165308A600A701640083120317100878
:10140800003C8A150A120313031D0F2A8A01B12210
:101418008A150A12112A8A01AD2283166908C307A0
:101428008A150A128312031CDB2983165208C3008B
:10143800831264008316430853028A150A12831222
:10144800031C5B2A83164308A600A7014F08A400C3
:10145800A5016400831203171008003C8A150A12BC
:101468000313031D3C2A8A01B1228A150A123E2A57
:101478008A01AD2283165008A400A50164008312D6
:1014880003171008003C8A150A120313031D512A7A
:101498008A01B1228A150A12532A8A01AD228316BB
:1014A8006908C3078A150A128312031C1D2A08003B
:1014B8008316D8015708D90083120230A600A70165
:1014C800831657088312A200A3018A01AD2183164F
:1014D800AE00831225088316AF002E08023CA80030
:1014E8002F08031C013E003CA900831264008316E8
:1014F800580859028A150A128312031CBE2A64006E
:1015080003171008003C8A150A120313031D912AB9
:101518008A01A2238A150A12932A8A011B24831698
:1015280059085802AE00AF01031CAF038312043000
:10153800A600A70183162E088312A20083162F087F
:101548008312A3008A01AD218316AE0083122508F9
:101558008316AF000A30AE070318AF0A2E08A80793
:101568002F080318013EA907D903D80A83128A1540
:101578000A127A2A08008316D8015708D90083125C
:101588000230A600A701831657088312A200A30100
:101598008A01AD218316AE00831225088316AF0099
:1015A8002E08023CA8002F08031C013E003CA9009D
:1015B800831264008316580859028A150A12831286
:1015C800031C152B640003171008003C8A150A1227
:1015D8000313031DF42A8A01A2238A150A12F62A84
:1015E8008A011B240430A600A70183165808831219
:1015F800A200A3018A01AD218316AE00831225083B
:101608008316AF000630AE070318AF0A2E08A807E6
:101618002F080318013EA907D80A83128A150A124F
:10162800DD2A08000730B6004030B4002030AA0098
:10163800AB01AE01AF010230A90083164008831246
:10164800A400A5019A30B000B1018A01DE2008008B
:101658000730B6008030B4002030AA00AB018A0100
:1016680069205D3C8A150A12031D332B0230A9003C
:101678006930B000B101A50158308A018A2083166B
:10168800C301831264000230831643028A150A12CA
:10169800831203185E2B8A150A12682083164308E2
:1016A800583E84005E088000C30A8A150A12831215
:1016B800031D462B5808A000A10104308A015821B7
:1016C8008316AE00831221088316AF0083125908CF
:1016D80083162E048312FF0008000730B6008030FE
:1016E800B4002030AA00AB018A0169205D3C8A154C
:1016F8000A12031D782B0430A9006930B000B1012B
:10170800A50158308A018A208316C3018312640018
:101718000430831643028A150A1283120318A32B76
:101728008A150A12682083164308583E84005E080A
:101738008000C30A8A150A128312031D8B2B5808CE
:10174800A000A10104308A0158218316AE0083123B
:1017580021088316AF008312590883162E048312BA
:10176800FF005A08A000A10104308A0158218316FD
:10177800AE00831221088316AF0083125B0883161C
:101788002E04B600831208000730B6008030B4007B
:101798002030AA00AB018A0169205D3C8A150A1233
:1017A800031DCF2B0630A9006930B000B101A50197
:1017B80058308A018A208316C301831264000630D8
:1017C800831643028A150A1283120318FA2B8A1504
:1017D8000A12682083164308583E84005E08800079
:1017E800C30A8A150A128312031DE22B5808A000A7
:1017F800A10104308A0158218316AE008312210802
:101808008316AF008312590883162E048312FF0033
:101818005A08A000A10104308A0158218316AE009D
:10182800831221088316AF0083125B0883162E04E7
:10183800B60083125C08A000A10104308A01582177
:101848008316AE00831221088316AF0083125D0849
:1018580083162E04B700831208000730B6008030C4
:10186800B4002030AA00AB018A0169205D3C8A15CA
:101878000A12031D382C8A0169208316DE003030D5
:101888005E02E9005E08C000831208000730B60057
:101898008030B4002030AA00AB018A0169205D3C89
:1018A8008A150A12031D512C0830A9006930B000AE
:1018B800B101A50158308A018A208316C301831219
:1018C80064000830831643028A150A12831203182B
:1018D8007C2C8A150A12682083164308583E840017
:1018E8005E088000C30A8A150A128312031D642C3D
:1018F8005808A000A10104308A0158218316AE00BF
:10190800831221088316AF008312590883162E0408
:10191800CF0083125A08A000A10104308A0158217F
:101928008316AE00831221088316AF0083125B086A
:1019380083162E04D00083125C08A000A101043095
:101948008A0158218316AE00831221088316AF003E
:1019580083125D0883162E04D20083125E08A0004D
:10196800A10104308A0158218316AE008312210890
:101978008316AF0083125F0883162E04D3008312E8
:1019880008007F088316D5003608D6003708D70028
:10199800831208007F088316A400A5013608A60054
:1019A800A701831208008A0194248A150A124B2081
:1019B8000D30F500F6010730B6001030B4000730DE
:1019C800B7000830B500A0308A01202076088A01C7
:1019D800202075088A0120208A0105208316BE0070
:1019E80064003E081F3C8A150A128312031D602DED
:1019F800F501F6018316A601A701831283162608AE
:101A08008312A000831627088312A100A3013F3088
:101A18008A016F218A150A12031D5A2D8316A40103
:101A2800A5018312831624088312A00083162508B3
:101A38008312A100A301EF308A016F218A150A12CF
:101A4800031D512D0730B6001030B4000730B70021
:101A58000830B500A0308A01202076088A012020AD
:101A680075088A0120208A0105208316BE0083128A
:101A78008A150A123720F50A0319F60A0830831660
:101A8800A4078A150A128312031C162D8316A50AA9
:101A98008A150A128312031D162D8316A60A031926
:101AA800A70A8A150A128312031D022D07141B3078
:101AB800A30058308A012F218A01C2248A150A12EC
:101AC8005E2083167730D5001F30D6000A30D70045
:101AD800831264001F30831657028A150A12831274
:101AE8000318802D8A0106250A308316D7078A1520
:101AF8000A128312031C6D2D83162D30D5001F305A
:101B0800D6000A30D700831264001F3083165702AC
:101B18008A150A12831203189C2D8A150A12BF22ED
:101B28000A308316D7078A150A128312031C882DD8
:101B38008316C230D5001F30D6000A30D700831272
:101B480064001F30831657028A150A12831203187D
:101B5800B82D8A150A125C220A308316D7078A150F
:101B68000A128312031CA42D0730A300D0308A0167
:101B78002F21031701309000831603132D30D50051
:101B88001F30D6000A30D700831264001F30831636
:101B980057028A150A1283120318DD2D8A150A12B4
:101BA800BF220A308316D7078A150A128312031C2C
:101BB800C92D0130A300F4308A012F218316773014
:101BC800D5001F30D6000A30D700831264001F30BA
:101BD800831657028A150A1283120318FD2D8A01EB
:101BE80006250A308316D7078A150A128312031CA2
:101BF800EA2D0130A300F4308A012F218316C23068
:101C0800D5001F30D6000A30D700831264001F3079
:101C1800831657028A150A12831203181E2E8A1574
:101C28000A125C220A308316D7078A150A12831211
:101C3800031C0A2E0317900103138A01C2248A1574
:101C48000A125E2083160830A400A5010830A600F9
:101C5800A701C301831264001B30831643028A154F
:101C68000A1283120318772E831643081A3C8A1522
:101C78000A128312031C6A2E8A150A124926831631
:101C8800BB0083128A150A126A2E0E308A00831648
:101C980043088312820753346834613472347034D1
:101CA80020343234343430347834363434342034D4
:101CB8007534733469346E346734203461342034B5
:101CC8005434363439343634333443348A0199271A
:101CD80008308316A4070318A50AC30A8A150A122E
:101CE8008312031D2F2E0730A300D0308A012F2125
:101CF80083162830A400A5011830A600A701C30147
:101D0800831264001330831643028A150A12831261
:101D18000318C52E83164308123C8A150A1283122B
:101D2800031CB82E8A150A129F268316BB0083123D
:101D38008A150A12B82E0E308A00831643088312B9
:101D48008207203442347934203443344F344D34BC
:101D58005034533479347334283463342934203478
:101D680032343034303437348A01992708308316B6
:101D7800A4070318A50AC30A8A150A128312031DA9
:101D8800852E83162230A600A7013030A400A501B5
:101D98008312831624088312A00083162508831251
:101DA800A100A301C8308A016F218A150A12031DF8
:101DB800F42E83162130A600A70183128A01B122CE
:101DC80083162330A600A70183128A01B122831645
:101DD800A40A0319A50A8A150A128312031DCD2E17
:101DE8000730A300D0308A012F218A0194248A1554
:101DF8000A125E2083160430E9000A30ED00323002
:101E0800EC000A30EB007830EA0083128A150A12D7
:101E180021218A150A12B42083162030A400A501B6
:101E2800A601A701C301831264000630831643028A
:101E38008A150A12831203184B2F83164308053C90
:101E48008A150A128312031C3E2F8A150A1232279A
:101E58008316BB0083128A150A123E2F0F308A00A0
:101E68008316430883128207533459345334543445
:101E780045344D348A01992708308316A40703187E
:101E8800A50AC30A8A150A128312031D182F83167E
:101E9800A401A5011030A600A701C30183126400A4
:101EA8000430831643028A150A1283120318842FFA
:101EB80083164308033C8A150A128312031C772FE2
:101EC8008A150A126D278316BB0083128A150A1217
:101ED800772F0F308A008316430883128207543401
:101EE80045344D3450348A01992708308316A607A3
:101EF8000318A70AC30A8A150A128312031D532F4F
:101F080083162030A400A5013830A600A701C3011C
:101F1800831264000630831643028A150A1283125C
:101F28000318C02F83164308053C8A150A1283122A
:101F3800031CB32F8A150A12A7278316BB00831226
:101F48008A150A12B32F0F308A00831643088312AA
:101F5800820748344F34553452344C3459348A014A
:101F6800992708308316A4070318A50AC30A8A15F7
:101F78000A128312031D8D2FFF3083166C07A600EB
:101F8800FF300318013EA7006B08A400A5018312C7
:101F9800831624088312A000831625088312A10043
:101FA80083166A0883128A016E218A110A16031D94
:101FB8003B287D08A0007E08A1008A01092120088D
:101FC800FD002108FE00640080307D028A150A1297
:101FD800031CF92F01308316A6020030031C013EB2
:101FE800A70283128A150A12FE2F8316A60A03195E
:101FF800A70A8312831626088312A00083162708CF
:102008008312A10083166C0883128A0172218A1137
:102018000A16031D1828FF3083166C07A600FF3028
:102028000318013EA7008312831626088312A00016
:10203800831627088312A10083166D0883128A016C
:102048006A218A110A16031D3028013083166D078C
:10205800A600A701A70D83128A01B1228316A40A3C
:102068000319A50A8A150A128312031DCC2F831699
:102078007A30A400A5011830A600A701C301831275
:1020880064000D30831643028A110A16831203185E
:102098007E28831643080C3C8A110A168312031CF7
:1020A80071288A110A165E208316BB0083128A11D2
:1020B8000A16712810308A00831643088312820793
:1020C8005434653472346D3469346E3461346C342C
:1020D80020344D346F34643465348A0199270830CC
:1020E8008316A4070318A50AC30A8A110A168312BD
:1020F800031D442883167830A400A5012030A600CB
:10210800A701C301831264000D30831643028A11AC
:102118000A1683120318C128831643080C3C8A1137
:102128000A168312031CB4288A110A16A1208316E2
:10213800BB0083128A110A16B42810308A0083164D
:10214800430883128207573461346934743469341C
:102158006E3467342E342E342E342E342E342E34EE
:102168008A01992708308316A4070318A50AC30A09
:102178008A110A168312031D872883167A30A40051
:10218800A5012830A600A701C301831264000E3000
:10219800831643028A110A16831203180529831627
:1021A80043080D3C8A110A168312031CF8288A1169
:1021B8000A16E4208316BB0083128A110A16F8282F
:1021C80010308A008316430883128207553473340B
:1021D8006534203447344C345534543449344C3401
:1021E800203431342E3433348A0199270830831649
:1021F800A4070318A50AC30A8A110A168312031D25
:10220800CA280730B6004030B4002030AA00AB011D
:10221800AE01AF0152308A019B2065308A019B20B4
:1022280061308A019B2064308A019B2079308A01C1
:102238009B203A308A019B200A308A019B200D306E
:102248008A019B200730B6008030B4002030AA00F5
:10225800AB018A0169205D3C8A110A16031D2D29EC
:102268008A0169208316DE005E088312A0006330AD
:102278008A0165218316AE005E088312A0004330F0
:102288008A0165218316B0002E0830048A110A16C7
:102298008312031D622B83165E088312A00073301D
:1022A8008A0165218316AE005E088312A0005330B0
:1022B8008A0165218316B0002E0830048A110A1697
:1022C8008312031D6D2B83165E088312A0007130E4
:1022D8008A0165218316AE005E088312A000513082
:1022E8008A0165218316B0002E0830048A110A1667
:1022F8008312031D792B83165E088312A0007430A5
:102308008A0165218316AE005E088312A00054304E
:102318008A0165218316B0002E0830048A110A1636
:102328008312031D852B83165E088312A0006C3070
:102338008A0165218316AE005E088312A0004C3026
:102348008A0165218316B0002E0830048A110A1606
:102358008312031DA82B83165E088312A000723017
:102368008A0165218316AE005E088312A0005230F0
:102378008A0165218316B0002E0830048A110A16D6
:102388008312031D9C2B83165E088312A000623003
:102398008A0165218316AE005E088312A0004230D0
:1023A8008A0165218316B0002E0830048A110A16A6
:1023B8008312031D902B83165E088312A0006B30D6
:1023C8008A0165218316AE005E088312A0004B3097
:1023D8008A0165218316B0002E0830048A110A1676
:1023E8008312031DD82B83165E088312A000643065
:1023F8008A0165218316AE005E088312A00044306E
:102408008A0165218316B0002E0830048A110A1645
:102418008312031DE12B83165E088312A00065302A
:102428008A0165218316AE005E088312A00045303C
:102438008A0165218316B0002E0830048A110A1615
:102448008312031DDD2B83165E088312A0007030F3
:102458008A0165218316AE005E088312A000503001
:102468008A0165218316B0002E0830048A110A16E5
:102478008312031DEF2B83165E088312A0007530AC
:102488008A0165218316AE005E088312A0005530CC
:102498008A0165218316B0002E0830048A110A16B5
:1024A8008312031D012C83165E088312A000783066
:1024B8008A0165218316AE005E088312A000583099
:1024C8008A0165218316B0002E0830048A110A1685
:1024D8008312031DB02B83165E088312A000793087
:1024E8008A0165218316AE005E088312A000593068
:1024F8008A0165218316B0002E0830048A110A1655
:102508008312031DC42B83165E088312A000663055
:102518008A0165218316AE005E088312A00046304A
:102528008A0165218316B0002E0830048A110A1624
:102538008312031D112C83165E088312A0006830D5
:102548008A0165218316AE005E088312A000483018
:102558008A0165218316B0002E0830048A110A16F4
:102568008312031D222C83165E088312A000763086
:102578008A0165218316AE005E088312A0005630DA
:102588008A0165218316B0002E0830048A110A16C4
:102598008312031D752C83165E088312A0006D300C
:1025A8008A0165218316AE005E088312A0004D30B3
:1025B8008A0165218316B0002E0830048A110A1694
:1025C8008312031DCA2D83165E088312A0006E3085
:1025D8008A0165218316AE005E088312A0004E3082
:1025E8008A0165218316B0002E0830048A110A1664
:1025F8008312031D812D83165E088312A0006F309D
:102608008A0165218316AE005E088312A0004F3050
:102618008A0165218316B0002E0830048A110A1633
:102628008312031DDC2C83165E088312A000613020
:102638008A0165218316AE005E088312A00041302E
:102648008A0165218316B0002E0830048A110A1603
:102658008312031DE22C83165E088312A0006730E4
:102668008A0165218316AE005E088312A0004730F8
:102678008A0165218316B0002E0830048A110A16D3
:102688008312031DD52C83165E088312A0007730B1
:102698008A0165218316AE005E088312A0005730B8
:1026A8008A0165218316B0002E0830048A110A16A3
:1026B8008312031DCE2C8A110A1605298A150A12BF
:1026C800C8238A150A12C5248A0106258A110A1602
:1026D80005298A150A12C8238A150A12C5248A15DB
:1026E8000A12BF228A110A1605298A150A12C82356
:1026F8008A150A12C5248A150A125C228A110A163A
:1027080005298A150A12C8238A150A12C5248A01BE
:1027180092258A110A1605298A150A124A248A1549
:102728000A1231248A150A1290218A110A160529DB
:102738008A150A124A248A150A1231248A150A129D
:10274800D5218A110A1605298A150A124A248A01EE
:10275800F5258A110A1605298A150A12C8237F0841
:102768008316EB003608EA003708ED0083128A1555
:102778000A1231248A150A1221218A110A160529FA
:102788008A150A12C8237F088316ED003608EC0064
:102798003708EB0083128A150A1231248A150A12A7
:1027A800B4208A110A1605298A01C2248A110A1638
:1027B800052983160130E80083128A150A1271234D
:1027C8008A150A12CE248A01B1228316E8018312DF
:1027D8008A110A1605298A150A1271238A150A12FE
:1027E800CE248A150A12312483164008BB008312AE
:1027F8008A0199278A110A1605298A150A12C823F7
:102808008A150A12CE2483163708BE0083128A1549
:102818000A1237208A110A1605298A150A12312444
:102828008316CF01EF30D000D2013F30D30083129E
:102838008A150A1290218A110A1605298A150A1280
:1028480071238A150A12CE248A0142278316510859
:10285800EE0083128A150A12312464008316400898
:10286800403C8A110A1683120319722C64008316DD
:1028780040083B3C8A110A168312031D4C2C831610
:102888002030BB0083128A0199278A110A16522C1C
:1028980083164008BB0083128A01992708308316E3
:1028A800A4070318A50A24088312A0008316250884
:1028B8008312A100A301EF308A0173218A110A163D
:1028C800031D6A2C83166E08D10083128A014227E1
:1028D8008A150A1231248A110A16312C8A110A160D
:1028E80005298A150A1271238A150A12CE2483161D
:1028F8002408EE002608EF0083128A0142278A1571
:102908000A123124640083164008403C8A110A16D2
:1029180083120319CB2C6400831640083B3C8A11B0
:102928000A168312031DA12C83162030BB008312C4
:102938008A0199278A110A16A72C83164008BB001A
:1029480083128A01992783166E08A400A50108300E
:10295800A6070318A70A26088312A00083162708CB
:102968008312A100A3013F308A0173218A110A163C
:10297800031DC32C83166F08A600A70183128A01C2
:1029880042278A150A1231248A110A16862C8A11BE
:102998000A16052983160230C20083128A110A1604
:1029A800E62C83160330C20083128A110A16E62C1D
:1029B8008316C20183128A110A16E62C8316013087
:1029C800C20083128A150A124A2483164F088312FA
:1029D800F200831650088312F100831652088312FE
:1029E800F400831653088312F3007108EF0072088D
:1029F800F0006F08A0007008A1007408A300730815
:102A08008A016F218A110A16031D7B2D6400831623
:102A18004208003C8A110A168312031D2D2D8A15BF
:102A28000A122C230730B6001030B4000730B70064
:102A38000830B500A0308A01202070088A012020C3
:102A48006F088A0120207F088A011E200A308A0127
:102A58002E21640083164208013C8A110A1683124B
:102A6800031D4F2D0730B6001030B4000730B700F3
:102A78000830B500A0308A01202070088A01202083
:102A88006F088A0120208A0105208316C00083125E
:102A98008A150A121623640083164208023C8A111A
:102AA8000A168312031D622D8A150A122C236F0839
:102AB80003178D0003137F088A0120216400831601
:102AC8004208033C8A110A168312031D742D6F08ED
:102AD8008A0118218316C00083128A150A12162348
:102AE800EF0A0319F00A8A110A16031DFD2C831632
:102AF800C20183128A110A1605298A150A124A2464
:102B080083165208A600A70183128316260883128B
:102B1800A000831627088312A10083165308831286
:102B28008A016E218A110A16031DC72D83164F08C4
:102B3800A400A5018312831624088312A00083161B
:102B480025088312A1008316500883128A016E217A
:102B58008A110A16031DBE2D8A01A7228A150A1298
:102B680016238316A40A0319A50A8A110A168312C2
:102B7800031D9F2D8316A60A0319A70A8A110A1690
:102B88008312031D892D8A110A1605298A150A122E
:102B98004A2483165208A600A70183128316260822
:102BA8008312A000831627088312A10083165308F6
:102BB80083128A016E218A110A16031D152E8316A7
:102BC8004F08A400A5018312831624088312A000CD
:102BD800831625088312A1008316500883128A01E0
:102BE8006E218A110A16031D0C2E8A150A122C232F
:102BF8007F088316BE0083128A150A1237208316AF
:102C0800A40A0319A50A8A110A168312031DE82DBE
:102C18008316A60A0319A70A8A110A168312031D26
:0A2C2800D22D63008A110A16152E42
:02400E00753FFC
:00000001FF
